:020000040000FA
:040000007CEF11F090
:0800080063EF0FF0D9CFE5FF13
:10001000E1CFD9FF00C0E5FF01C0E5FF02C0E5FF69
:1000200003C0E5FF04C0E5FF05C0E5FF06C0E5FF2E
:1000300007C0E5FF08C0E5FF09C0E5FF0AC0E5FF0E
:100040000BC0E5FF0CC0E5FF0DC0E5FF0EC0E5FFEE
:100050000FC0E5FF10C0E5FF11C0E5FF12C0E5FFCE
:1000600013C0E5FF14C0E5FF020EDBCF00F0030E66
:10007000DBCF01F0040EDBCF02F0050EDBCF03F087
:10008000060EDBCF04F0070EDBCF05F0080EDBCF4A
:1000900006F0090EDBCF07F00A0EDBCF08F00B0EDF
:1000A000DBCF09F00C0EDBCF0AF00D0EDBCF0BF02F
:1000B0000001AD6B60AE29D0A49074AE13D009C01E
:1000C000E9FF0AC0F3FF0B5051EC11F00C6E0C86E7
:1000D0000CC0E5FF09C0E9FF0AC0F3FF0B5094EC28
:1000E00011F0749E0C6A60B00C2A0C50010BF46E77
:1000F0000001AD51FE0BF4100001AD6F0F0E0D6E3F
:10010000600E0C6E800E0E6E40D00F0150AF3BD0D3
:10011000A49274AC13D009C0E9FF0AC0F3FF0B50DE
:1001200051EC11F00F6E0F860FC0E5FF09C0E9FF1B
:100130000AC0F3FF0B5094EC11F0749C070E0F01F2
:1001400050150F6E0F500001AD6FADC0E8FF020EED
:100150000F5C12E209C0E9FF0AC0F3FF0B5051EC3B
:1001600011F00F6E0F8E0FC0E5FF09C0E9FF0AC046
:10017000F3FF0B5094EC11F00F0E0D6E500E0C6E41
:10018000800E0E6E02D0E86AFFD00CC00FF00DC0DA
:1001900010F00EC011F0000EE56E09C0E9FF0AC0B4
:1001A000F3FF0B5094EC11F00C50050F126E000E83
:1001B0000D20136E000E0E20146E12C0E9FF13C046
:1001C000F3FF145051EC11F0126E12500001AE6F9B
:1001D000AEC0E8FF0F0E121612C0E5FF06C0E9FF21
:1001E00007C0F3FF085094EC11F00001AEAD12D03F
:1001F00009C0E9FF0AC0F3FF0B5051EC11F0126E79
:10020000128C12C0E5FF09C0E9FF0AC0F3FF0B50D2
:1002100094EC11F00C50020F126E000E0D20136EB4
:10022000000E0E20146E12C0E9FF13C0F3FF14502D
:1002300051EC11F0126E12500001AE6F0001AEA72A
:1002400016D009C0E9FF0AC0F3FF0B5051EC11F0C2
:10025000126E128A12C0E5FF09C0E9FF0AC0F3FF5F
:100260000B5094EC11F0010E0001AE6F02D00001B2
:10027000AE6B0C50010F126E000E0D20136E000EAF
:100280000E20146E0001AE51E56E0250E56E015075
:10029000E56E0050E56E1450E56E1350E56E125099
:1002A000E56EB3EC06F0070EE126060E0C26000EF6
:1002B0000D22000E0E2206C0E9FF07C0F3FF085012
:1002C00051EC11F0066E06500001AE6F0CC000F04C
:1002D0000DC001F00EC002F0066A06C007F0086A01
:1002E00006BE0868AEC00CF00D6A0850800FF36EB1
:1002F0000D50800FF35C02E10C50075C1DE200C062
:10030000E9FF01C0F3FF025051EC11F0076E002A23
:10031000D8B0012AD8B0022A07C0E5FF03C0E9FF20
:1003200004C0F3FF055094EC11F0032AD8B0042A5E
:10033000D8B0052A062AD1D7A4AE13D009C0E9FF48
:100340000AC0F3FF0B5051EC11F0006E008800C0A2
:10035000E5FF09C0E9FF0AC0F3FF0B5094EC11F070
:10036000A49E0FC0E9FF10C0F3FF115051EC11F033
:10037000006E009E00C0E5FF0FC0E9FF10C0F3FF54
:10038000115094EC11F0010EE4CF14F0E4CF13F00F
:10039000E4CF12F0E4CF11F0E4CF10F0E4CF0FF08F
:1003A000E4CF0EF0E4CF0DF0E4CF0CF0E4CF0BF08F
:1003B000E4CF0AF0E4CF09F0E4CF08F0E4CF07F08F
:1003C000E4CF06F0E4CF05F0E4CF04F0E4CF03F08F
:1003D000E4CF02F0E4CF01F0E4CF00F0E4CFD9FFA6
:1003E0001200D9CFE5FFE1CFD9FF00C0E5FF01C082
:1003F000E5FF02C0E5FF03C0E5FF04C0E5FF05C05F
:10040000E5FF06C0E5FF07C0E5FF08C0E5FF09C03E
:10041000E5FF0AC0E5FF0BC0E5FF0CC0E5FF0DC01E
:10042000E5FF0EC0E5FF0FC0E5FF020EDBCF00F0D9
:10043000030EDBCF01F0040EDBCF02F0800EE56E81
:100440000BEC11F0E12A0F0E046E180E036E800EF5
:10045000056E000EE56E000EE56E000EE56E070EF1
:10046000E56EFF0EE56E0550E56E0450E56E035037
:10047000E56E1BEC08F0080EE1260F0E046E1C0E54
:10048000036E800E056E000EE56E000EE56E000E2A
:10049000E56E070EE56EFF0EE56E0550E56E045045
:1004A000E56E0350E56E1BEC08F0080EE126036ACA
:1004B000046A056A066A0450800F800F02E1060E86
:1004C000035CD8B04BD105500024076E06500120C4
:1004D000086EE86A06BEE8680220096E07C0E9FFF8
:1004E00008C0F3FF095027EC11F0076EF3CF08F0B6
:1004F0000750FF0A04E10850FF0A01E12FD1830EE3
:100500000324096E000E04200A6E09C0E9FF0AC028
:10051000EAFFEFCF09F0060E095CD8B0F9D010C0A1
:10052000E5FF11C0E5FF116A09341136E8341136D0
:10053000FC0B106E000EFB6E050EFA6E540E1026AC
:100540001150FA22D8B0FB2A1050E4CF11F0E4CFBA
:1005500010F0F96EB6EF02F0D9EF02F0FCEF02F006
:100560001FEF03F042EF03F065EF03F00D01D481BC
:100570000F0E0A6E000E096E800E0B6E07C00CF097
:1005800008C00DF00E6A0F6A000EE56E0F50E56EA2
:100590000E50E56E0D50E56E0C50E56E0B50E56E9D
:1005A0000A50E56E0950E56E1BEC08F0080EE126D6
:1005B000CDD00D01D4830F0E0A6E040E096E800E8D
:1005C0000B6E07C00CF008C00DF00E6A0F6A000E2B
:1005D000E56E0F50E56E0E50E56E0D50E56E0C5059
:1005E000E56E0B50E56E0A50E56E0950E56E1BECAA
:1005F00008F0080EE126AAD00D01D4850F0E0A6E70
:10060000080E096E800E0B6E07C00CF008C00DF0CE
:100610000E6A0F6A000EE56E0F50E56E0E50E56E25
:100620000D50E56E0C50E56E0B50E56E0A50E56E10
:100630000950E56E1BEC08F0080EE12687D00D018D
:10064000D4870F0E0A6E0C0E096E800E0B6E07C05B
:100650000CF008C00DF00E6A0F6A000EE56E0F5028
:10066000E56E0E50E56E0D50E56E0C50E56E0B50CC
:10067000E56E0A50E56E0950E56E1BEC08F0080EB9
:10068000E12664D00D01D4890F0E0A6E100E096E9A
:10069000800E0B6E07C00CF008C00DF00E6A0F6ADA
:1006A000000EE56E0F50E56E0E50E56E0D50E56ED6
:1006B0000C50E56E0B50E56E0A50E56E0950E56E84
:1006C0001BEC08F0080EE12641D00D01D48B0F0E73
:1006D0000A6E140E096E800E0B6E07C00CF008C077
:1006E0000DF00E6A0F6A000EE56E0F50E56E0E50AB
:1006F000E56E0D50E56E0C50E56E0B50E56E0A5040
:10070000E56E0950E56E1BEC08F0080EE1261ED0E0
:100710000D01D48B0F0E0A6E140E096E800E0B6E37
:100720000C6A0D6A000EE56E0D50E56E0C50E56E1C
:100730000850E56E0750E56E0B50E56E0A50E56E09
:100740000950E56E1BEC08F0080EE126020E0526A6
:10075000D8B0062A032AD8B0042AADD6000EE56E1A
:100760000BEC11F0E12AF36AE86AE4CF0FF0E4CF72
:100770000EF0E4CF0DF0E4CF0CF0E4CF0BF0E4CFBB
:100780000AF0E4CF09F0E4CF08F0E4CF07F0E4CFBB
:1007900006F0E4CF05F0E4CF04F0E4CF03F0E4CFBB
:1007A00002F0E4CF01F0E4CF00F0E4CFD9FF120073
:1007B000D9CFE5FFE1CFD9FF00C0E5FF01C0E5FFDC
:1007C00002C0E5FF03C0E5FF04C0E5FF05C0E5FF8B
:1007D00006C0E5FF07C0E5FF08C0E5FF09C0E5FF6B
:1007E0000AC0E5FF0BC0E5FF0CC0E5FF0DC0E5FF4B
:1007F0000EC0E5FF0FC0E5FF10C0E5FF11C0E5FF2B
:1008000012C0E5FF13C0E5FF14C0E5FF15C0E5FF0A
:10081000020EDBCF00F0030EDBCF01F0040EDBCFC6
:1008200002F0050EDBCF03F0060EDBCF04F0070E5F
:10083000DBCF05F0080EDBCF06F0090EDBCF07F0AB
:100840000A0EDBCF08F00F0E0A6E400E096E800E06
:100850000B6E09500001606F0A500001616F0B5070
:100860000001626F0F0E0A6E300E096E800E0B6E65
:1008700009500001636F0A500001646F0B500001C2
:10088000656F0F0E0A6E200E096E800E0B6E0950FA
:100890000001666F0A500001676F0B500001686F1E
:1008A000096A0A6A020E095CD8B0C5D0600E0A2433
:1008B0000B6E0C6A000E0C220BC0E9FF0CC0EAFFA5
:1008C000EECF0BF0EECF0CF0EFCF0DF00BC00EF033
:1008D0000CC00FF00DC010F00BC0E9FF0CC0F3FF0F
:1008E0000D5051EC11F0116E11B6A1D0FC0E111685
:1008F00011C0E5FF0BC0E9FF0CC0F3FF0D5094ECF5
:1009000011F00BC0E9FF0CC0F3FF0D5051EC11F0DA
:10091000116E030E0814126E1250111211C0E5FF71
:100920000BC0E9FF0CC0F3FF0D5094EC11F008ACC4
:1009300004D0400E0710116E02D007C011F00B500A
:10094000050F126E000E0C20136E000E0D20146E9B
:1009500011C0E5FF12C0E9FF13C0F3FF145094EC7F
:1009600011F008AA03D0010E116E01D0116A0B50CC
:10097000010F126E000E0C20136E000E0D20146E6F
:100980001150E56E0350E56E0250E56E0150E56EC4
:100990000050E56E1450E56E1350E56E1250E56E92
:1009A0001BEC08F0080EE126060E0B26000E0C22AA
:1009B000000E0D2204C011F005C012F006C013F0A5
:1009C000146A0750145C1DE211C0E9FF12C0F3FF66
:1009D000135051EC11F0156E112AD8B0122AD8B06C
:1009E000132A15C0E5FF0BC0E9FF0CC0F3FF0D5043
:1009F00094EC11F00B2AD8B00C2AD8B00D2A142A86
:100A0000E0D70EC0E9FF0FC0F3FF105051EC11F01A
:100A10000B6E0BB40AD00B860BC0E5FF0EC0E9FFCE
:100A20000FC0F3FF105094EC11F0010E05D0030E2F
:100A30000A26092A37D7E86AE4CF15F0E4CF14F084
:100A4000E4CF13F0E4CF12F0E4CF11F0E4CF10F0D4
:100A5000E4CF0FF0E4CF0EF0E4CF0DF0E4CF0CF0D4
:100A6000E4CF0BF0E4CF0AF0E4CF09F0E4CF08F0D4
:100A7000E4CF07F0E4CF06F0E4CF05F0E4CF04F0D4
:100A8000E4CF03F0E4CF02F0E4CF01F0E4CF00F0D4
:100A9000E4CFD9FF1200D9CFE5FFE1CFD9FF00C0E5
:100AA000E5FF01C0E5FF02C0E5FF03C0E5FF04C0AC
:100AB000E5FF05C0E5FF06C0E5FF07C0E5FF08C08C
:100AC000E5FF09C0E5FF0AC0E5FF0BC0E5FF0CC06C
:100AD000E5FF0DC0E5FF0EC0E5FF020EDBCF00F025
:100AE000030EDBCF01F0040EDBCF02F0050EDBCFEF
:100AF00003F0060EDBCF04F000500110D8A4EAD0BA
:100B000002C0E9FF03C0F3FF045027EC11F0056EAB
:100B1000F3CF06F00650E56E0550E56E000EE56E6B
:100B2000020EE56EF6EC0DF0076EF3CF08F0040E42
:100B3000E126096A0A6A400E07264B0E08224C0E6F
:100B40000922000E0A2205C00BF006C00CF00D6A47
:100B50000E6A0E50E56E0D50E56E0C50E56E0B50B2
:100B6000E56E0A50E56E0950E56E0850E56E0750D7
:100B7000E56E65EC09F0076EF3CF08F0F4CF09F0ED
:100B8000E9CF0AF0080EE126000EE56E000EE56ED4
:100B9000000EE56E040EE56E0A50E56E0950E56E36
:100BA0000850E56E0750E56E65EC09F0076EF3CF6F
:100BB00008F0F4CF09F0E9CF0AF0080EE126FF0EA5
:100BC0000726FF0E0822FF0E0922FF0E0A220A50F6
:100BD000800F800F08E1000E095C05E1010E085C42
:100BE00002E1000E075C0AE20850E56E0750E56E70
:100BF0003C0E20EC0FF0020EE12664D00650E56EAC
:100C00000550E56E000EE56E080EE56EF6EC0DF093
:100C1000056EF3CF06F0040EE126096A0A6A400E5B
:100C200005264B0E06224C0E0922000E0A220E50FB
:100C3000E56E0D50E56E0C50E56E0B50E56E0A50FA
:100C4000E56E0950E56E0650E56E0550E56E65EC03
:100C500009F0056EF3CF06F0F4CF09F0E9CF0AF002
:100C6000080EE126000EE56E000EE56E000EE56E44
:100C7000100EE56E0A50E56E0950E56E0650E56E01
:100C80000550E56E65EC09F0056EF3CF06F0F4CF84
:100C900009F0E9CF0AF0080EE126FF0E0526FF0E47
:100CA0000622FF0E0922FF0E0A220550076E06508B
:100CB000086E0850E56E0750E56E2C0E20EC0FF024
:100CC000020EE1260D0EA6EC11F0AB8EAB88F36A96
:100CD000010E28D00050010A02E1015001E020D0AD
:100CE000040E0226000E0322000E042202C0E9FFB9
:100CF00003C0F3FF045051EC11F0026E025007E004
:100D0000949A94889496C76A210EC66E06D0949AD7
:100D100094889486C76A250EC66EF36A010E02D0C7
:100D2000F36AE86AE4CF0EF0E4CF0DF0E4CF0CF004
:100D3000E4CF0BF0E4CF0AF0E4CF09F0E4CF08F001
:100D4000E4CF07F0E4CF06F0E4CF05F0E4CF04F001
:100D5000E4CF03F0E4CF02F0E4CF01F0E4CF00F001
:100D6000E4CFD9FF1200D9CFE5FFE1CFD9FF00C012
:100D7000E5FF01C0E5FF02C0E5FF03C0E5FF04C0D9
:100D8000E5FF05C0E5FF06C0E5FF07C0E5FF08C0B9
:100D9000E5FF09C0E5FF0AC0E5FF0BC0E5FF0CC099
:100DA000E5FF0DC0E5FF020EDBCF00F0030EDBCF49
:100DB00001F0040EDBCF02F0050EDBCF03F0060ED0
:100DC000DBCF04F0070EDBCF05F0080EDBCF06F01B
:100DD0000650D8A46CD000C0E9FF01C0F3FF025058
:100DE00051EC11F0066E0638E840F80B076E07C0AC
:100DF000E5FF03C0E9FF04C0F3FF055094EC11F0D8
:100E00000350010F086E000E0420096E000E05202D
:100E10000A6E0638E840070B066E06C0E5FF08C0FC
:100E2000E9FF09C0F3FF0A5094EC11F0002AD8B092
:100E3000012AD8B0022A00C0E9FF01C0F3FF025026
:100E400051EC11F0066E0638E840070B066E0650AE
:100E5000071207C0E5FF03C0E9FF04C0F3FF055018
:100E600094EC11F00350020F066E000E0420076E82
:100E7000000E0520086E000EE56E06C0E9FF07C0F3
:100E8000F3FF085094EC11F00350030F066E000EB0
:100E90000420076E000E0520086E000EE56E06C0E9
:100EA000E9FF07C0F3FF085094EC11F0A5D0035000
:100EB000020F066E000E0420076E000E0520086E5D
:100EC00000C0E9FF01C0F3FF025051EC11F0096EC0
:100ED0000938E844E00B0A6E0AC0E5FF06C0E9FFE6
:100EE00007C0F3FF085094EC11F00350030F0B6E92
:100EF000000E04200C6E000E05200D6E0938E8442B
:100F00001F0B096E09C0E5FF0BC0E9FF0CC0F3FF22
:100F10000D5094EC11F0002AD8B0012AD8B0022A62
:100F200006C0E9FF07C0F3FF085051EC11F0E86E6E
:100F300000C0E9FF01C0F3FF025051EC11F0096E4F
:100F4000030E09140B6E0B500A120AC0E5FF06C00F
:100F5000E9FF07C0F3FF085094EC11F006C0E9FF69
:100F600007C0F3FF085051EC11F0E86EE00E0916CF
:100F70000938E8441F0B096E09500A120AC0E5FF40
:100F800006C0E9FF07C0F3FF085094EC11F0002AF7
:100F9000D8B0012AD8B0022A0350010F066E000E05
:100FA0000420076E000E0520086E00C0E9FF01C096
:100FB000F3FF025051EC11F0096E09C0E5FF06C0C5
:100FC000E9FF07C0F3FF085094EC11F0002AD8B0F5
:100FD000012AD8B0022A00C0E9FF01C0F3FF025085
:100FE00051EC11F0006E00C0E5FF03C0E9FF04C042
:100FF000F3FF055094EC11F0E4CF0DF0E4CF0CF0CA
:10100000E4CF0BF0E4CF0AF0E4CF09F0E4CF08F02E
:10101000E4CF07F0E4CF06F0E4CF05F0E4CF04F02E
:10102000E4CF03F0E4CF02F0E4CF01F0E4CF00F02E
:10103000E4CFD9FF1200D9CFE5FFE1CFD9FF00C03F
:10104000E5FF01C0E5FF02C0E5FF03C0E5FF04C006
:10105000E5FF05C0E5FF06C0E5FF07C0E5FF08C0E6
:10106000E5FF09C0E5FF0AC0E5FF020EDBCF00F097
:10107000030EDBCF01F0040EDBCF02F0050EDBCF59
:10108000A0F0060EDBCFA1F0070EDBCFA2F0080E1A
:10109000DBCFA3F0090EDBCF03F0000E056EA00E30
:1010A000046E800E066E0350D8A450D004C0E9FF31
:1010B00005C0F3FF065051EC11F0036E0338E8440D
:1010C0001F0B076E07C0E5FF00C0E9FF01C0F3FF7B
:1010D000025094EC11F000C0E9FF01C0F3FF025090
:1010E00051EC11F0076E0450010F086E000E052040
:1010F000096E000E06200A6E08C0E9FF09C0F3FF62
:101100000A5051EC11F0086E0838E844E00B096E03
:101110000950071207C0E5FF00C0E9FF01C0F3FF57
:10112000025094EC11F0002AD8B0012AD8B0022A5B
:101130000338E844E00B076E07C0E5FF00C0E9FF95
:1011400001C0F3FF025094EC11F0A6D00450020F3E
:10115000036E000E0520076E000E0620086E03C009
:10116000E9FF07C0F3FF085051EC11F0036E03389C
:10117000E840070B076E07C0E5FF00C0E9FF01C0AC
:10118000F3FF025094EC11F000C0E9FF01C0F3FF3F
:10119000025051EC11F0076E0450030F086E000E60
:1011A0000520096E000E06200A6E08C0E9FF09C07E
:1011B000F3FF0A5051EC11F0086E0838E840F80BC4
:1011C000096E0950071207C0E5FF00C0E9FF01C022
:1011D000F3FF025094EC11F0002AD8B0012AD8B0E5
:1011E000022A0338E840F80B076EE00E071607C026
:1011F000E5FF00C0E9FF01C0F3FF025094EC11F0DD
:10120000078607C0E5FF00C0E9FF01C0F3FF0250F9
:1012100094EC11F0030E03160350071207C0E5FF0C
:1012200000C0E9FF01C0F3FF025094EC11F0002A66
:10123000D8B0012AD8B0022A0450010F036E000E64
:101240000520076E000E0620086E03C0E9FF07C0E8
:10125000F3FF085051EC11F0036E03C0E5FF00C02E
:10126000E9FF01C0F3FF025094EC11F0002AD8B05E
:10127000012AD8B0022A04C0E9FF05C0F3FF0650D6
:1012800051EC11F0046E04C0E5FF00C0E9FF01C09D
:10129000F3FF025094EC11F0E4CF0AF0E4CF09F030
:1012A000E4CF08F0E4CF07F0E4CF06F0E4CF05F098
:1012B000E4CF04F0E4CF03F0E4CF02F0E4CF01F098
:1012C000E4CF00F0E4CFD9FF1200D9CFE5FFE1CFA2
:1012D000D9FF00C0E5FF01C0E5FF02C0E5FF03C084
:1012E000E5FF04C0E5FF05C0E5FF06C0E5FF07C058
:1012F000E5FF08C0E5FF09C0E5FF0AC0E5FF0BC038
:10130000E5FF0CC0E5FF0DC0E5FF020EDBCF00F0EE
:10131000030EDBCF01F0040EDBCF02F0050EDBCFB6
:1013200003F0060EDBCF04F0070EDBCF05F0080E4E
:10133000DBCF06F0090EDBCF07F0D88003AED890E4
:10134000086A083608500FE0031C0C6E021C0B6E76
:10135000011C0A6E001C096E092A0DE10A2A0BE124
:101360000B4A0C2A08D000C009F001C00AF002C0E4
:101370000BF003C00CF009C000F00AC001F00BC074
:1013800002F00CC003F0D88007AED890096A093685
:1013900009500FE0071C0D6E061C0C6E051C0B6E31
:1013A000041C0A6E0A2A0DE10B2A0BE10C4A0D2AD5
:1013B00008D004C00AF005C00BF006C00CF007C04E
:1013C0000DF00D50E56E0C50E56E0B50E56E0A50B9
:1013D000E56E0350E56E0250E56E0150E56E00507B
:1013E000E56EADEC0BF0006EF3CF01F0F4CF02F040
:1013F000E9CF03F0080EE1260950081A085016E05C
:10140000031C076E021C066E011C056E001C046E98
:10141000042A04E1052A02E1064A072A07C0E9FF77
:1014200006C0F4FF05C0F3FF045007D003C0E9FF76
:1014300002C0F4FF01C0F3FF0050E4CF0DF0E4CF91
:101440000CF0E4CF0BF0E4CF0AF0E4CF09F0E4CFE6
:1014500008F0E4CF07F0E4CF06F0E4CF05F0E4CFE6
:1014600004F0E4CF03F0E4CF02F0E4CF01F0E4CFE6
:1014700000F0E4CFD9FF1200D9CFE5FFE1CFD9FFCB
:1014800000C0E5FF01C0E5FF02C0E5FF03C0E5FFC6
:1014900004C0E5FF05C0E5FF06C0E5FF07C0E5FFA6
:1014A00008C0E5FF09C0E5FF0AC0E5FF0BC0E5FF86
:1014B0000CC0E5FF0DC0E5FF0EC0E5FF020EDBCF5F
:1014C00000F0030EDBCF01F0040EDBCF02F0000EC4
:1014D000046E9C0E036E800E056E0050030F066EA8
:1014E000000E0120076E000E0220086E0050020F51
:1014F000096E000E01200A6E000E02200B6E000E17
:101500000D6EAC0E0C6E800E0E6E0E50E56E0D5014
:10151000E56E0C50E56E0B50E56E0A50E56E095015
:10152000E56E0850E56E0750E56E0650E56E055015
:10153000E56E0450E56E0350E56E06EC00F0036EB8
:101540000C0EE126035003E1F36AE86A42D0000181
:101550009C51036E00019D51046E03C0E5FF04C061
:10156000F4FF00C0E9FF01C0F3FF025088EC11F066
:1015700099C003F0032A03500001996F0001AC5198
:10158000600B09E09BC003F0032A035000019B6F2E
:10159000F368E8681ED00001ACA709D09AC003F038
:1015A000032A035000019A6FF368FE0E12D0020E58
:1015B0000026000E0122000E022200C0E9FF01C039
:1015C000F3FF025051EC11F0006E016A01C0F3FF0D
:1015D0000050E4CF0EF0E4CF0DF0E4CF0CF0E4CFF8
:1015E0000BF0E4CF0AF0E4CF09F0E4CF08F0E4CF49
:1015F00007F0E4CF06F0E4CF05F0E4CF04F0E4CF49
:1016000003F0E4CF02F0E4CF01F0E4CF00F0E4CF48
:10161000D9FF12000001A46B060E0001A56F0001A6
:101620008B6BE10E00018C6F010E00018E6F010EBD
:101630000001956F000E016E8B0E006E800E026E23
:101640000250E56E0150E56E0050E56E000EE56E4D
:10165000000EE56E4BEC05F0050EE126000E016E66
:10166000910E006E800E026E0250E56E0150E56E26
:101670000050E56E000EE56E010EE56E4BEC05F0D8
:10168000050EE126000E016EA40E006E800E026EA5
:101690000250E56E0150E56E0050E56E000EE56EFD
:1016A00042EC0DF0040EE12670EC11F0FC0E9316E6
:1016B0008A828A90E86AE86A010E006E016A000E6A
:1016C000E56E010EE56E9AEC10F0026E020EE12658
:1016D000025015E0000EE56E010EE56E6DEC10F0A7
:1016E0000001896F020EE12600018951E56E000EAE
:1016F000E56E000EE56E3AEC10F0030EE126000EEA
:10170000E56E000EE56E9AEC10F0026E020EE12618
:101710000250010A13E1000EE56E000EE56E6DEC5D
:1017200010F0026E020EE1260250E56E000EE56E2C
:10173000010EE56E3AEC10F0030EE126002AD8B057
:10174000012A0150800F460F02E1990E005C02E36E
:101750008A80B5D78A90B3D71200D9CFE5FFE1CF01
:10176000D9FF00C0E5FF01C0E5FF02C0E5FF03C0EF
:10177000E5FF04C0E5FF05C0E5FF06C0E5FF07C0C3
:10178000E5FF08C0E5FF09C0E5FF0AC0E5FF0BC0A3
:10179000E5FF0CC0E5FF0DC0E5FF020EDBCF00F05A
:1017A000030EDBCF01F0040EDBCF02F0050EDBCF22
:1017B00003F0060EDBCF04F0070EDBCF05F0080EBA
:1017C000DBCF06F0090EDBCF07F0086A096A0A6A68
:1017D0000B6A200E0C6E0344010B0D6E010E0D16EC
:1017E0000050002601360236033608500826093616
:1017F0000A360B360D50D8A4088007500B5C08E160
:1018000006500A5C05E10550095C02E10450085CE1
:1018100009E30450085E0550095A06500A5A075059
:101820000B5A00800C2ED7D703C0E9FF02C0F4FF8B
:1018300001C0F3FF0050E4CF0DF0E4CF0CF0E4CF93
:101840000BF0E4CF0AF0E4CF09F0E4CF08F0E4CFE6
:1018500007F0E4CF06F0E4CF05F0E4CF04F0E4CFE6
:1018600003F0E4CF02F0E4CF01F0E4CF00F0E4CFE6
:10187000D9FF1200D9CFE5FFE1CFD9FF00C0E5FFC6
:1018800001C0E5FF02C0E5FF03C0E5FF04C0E5FFBE
:1018900005C0E5FF06C0E5FF07C0E5FF08C0E5FF9E
:1018A00009C0E5FF020EDBCF00F0030EDBCF01F035
:1018B000040EDBCF02F000C0E9FF01C0F3FF0250CD
:1018C00027EC11F0036EF3CF04F0056A066A0050AE
:1018D000030F076E000E0120086E000E0220096E35
:1018E000020E0026000E0122000E022200C0E9FFB7
:1018F00001C0F3FF025051EC11F0006E000EE56ED6
:101900000050E56E0950E56E0850E56E0750E56E33
:101910000650E56E0550E56E0450E56E0350E56E29
:10192000D8EC03F0006E090EE126016A00500110A8
:1019300007E097C002F0022A02500001976F06D01C
:1019400098C002F0022A02500001986F01C0F3FF14
:101950000050E4CF09F0E4CF08F0E4CF07F0E4CF83
:1019600006F0E4CF05F0E4CF04F0E4CF03F0E4CFD9
:1019700002F0E4CF01F0E4CF00F0E4CFD9FF120091
:10198000D9CFE5FFE1CFD9FF00C0E5FF01C0E5FFFA
:1019900002C0E5FF03C0E5FF04C0E5FF05C0E5FFA9
:1019A00006C0E5FF07C0E5FF08C0E5FF09C0E5FF89
:1019B0000AC0E5FF0BC0E5FF020EDBCF00F0030E0F
:1019C000DBCF01F0040EDBCF02F0050EDBCF03F01E
:1019D000060EDBCF04F0070EDBCF05F0080EDBCFE1
:1019E00006F00050011006E00050010A02E101502B
:1019F00001E02DD0076A086A0850800FF36E065088
:101A0000800FF35C02E10550075C21E207500224DD
:101A1000096E085003200A6EE86A08BEE8680420D0
:101A20000B6E09C0E9FF0AC0F3FF0B5051EC11F037
:101A3000096E0950E56E0150E56E0050E56E3AEC16
:101A400010F0030EE126072AD8B0082AD5D7E4CF34
:101A50000BF0E4CF0AF0E4CF09F0E4CF08F0E4CFD4
:101A600007F0E4CF06F0E4CF05F0E4CF04F0E4CFD4
:101A700003F0E4CF02F0E4CF01F0E4CF00F0E4CFD4
:101A8000D9FF1200D9CFE5FFE1CFD9FF00C0E5FFB4
:101A900001C0E5FF02C0E5FF03C0E5FF020EDBCF9A
:101AA00000F0030EDBCF01F0040EDBCF02F0050ED9
:101AB000DBCF03F0030E005CD8B03CD004C0E5FFE0
:101AC00005C0E5FF056A00340536E8340536FC0B31
:101AD000046E000EFB6E1A0EFA6EF20E042605500E
:101AE000FA22D8B0FB2A0450E4CF05F0E4CF04F08A
:101AF000F96E7FEF0DF09AEF0DF09AEF0DF0012ADD
:101B0000D8B0022AD8B0032A01C0E9FF02C0F3FF0F
:101B1000035051EC11F0006E080E005C09E2D56A2A
:101B2000800ED510016E00500110D56E010E03D04D
:101B3000E86A01D0E86AE4CF03F0E4CF02F0E4CF32
:101B400001F0E4CF00F0E4CFD9FF1200D9CFE5FFD8
:101B5000E1CFD9FF00C0E5FF01C0E5FF02C0E5FF0E
:101B600003C0E5FF04C0E5FF05C0E5FF06C0E5FFD3
:101B700007C0E5FF020EDBCF00F0030EDBCF01F064
:101B8000040EDBCF02F0050EDBCF03F0060EDBCF39
:101B900004F0056A0450055C15E205500024066E49
:101BA00001C0E9FF02C0F3FF035051EC11F0076ED2
:101BB0000750E56E0650E56E9BEC0FF0020EE12635
:101BC000052AE8D70450E4CF07F0E4CF06F0E4CFCD
:101BD00005F0E4CF04F0E4CF03F0E4CF02F0E4CF6B
:101BE00001F0E4CF00F0E4CFD9FF1200D9CFE5FF38
:101BF000E1CFD9FF00C0E5FF01C0E5FF02C0E5FF6E
:101C000003C0E5FF020EDBCF00F0030EDBCF01F0D7
:101C1000040EDBCF02F0050EDBCF03F00050000115
:101C2000A66F0150A76F02500001A86F0350A96F63
:101C30000001A6510001A803F3CF00F0F4CF01F09A
:101C400000500001AA6F0150AB6F0001A6510001C6
:101C5000A903F3CF00F00001A7510001A803F3CFBF
:101C600001F0015000260001AB5100260050AB6F7F
:101C7000ABC0F3FFAA51E4CF03F0E4CF02F0E4CF0E
:101C800001F0E4CF00F0E4CFD9FF1200A20EF66E0F
:101C9000230EF76E000EF86E0900F550056E090070
:101CA000F550066E055002E106503BE00900F55084
:101CB000006E0900F550016E0900F550026E090032
:101CC0000900F550E96E0900F550EA6E09000900B7
:101CD0000900F550036E0900F550046E0900090073
:101CE000F6CF07F0F7CF08F0F8CF09F000C0F6FF05
:101CF00001C0F7FF02C0F8FF035002E1045007E003
:101D00000900F550EE6E0306F8E20406F9D707C0A5
:101D1000F6FF08C0F7FF09C0F8FF0506C4E2060693
:101D2000C5D71200D9CFE5FFE1CFD9FF00C0E5FF4D
:101D300001C0E5FF02C0E5FF03C0E5FF04C0E5FF09
:101D400005C0E5FF06C0E5FF020EDBCF00F0030E85
:101D5000DBCF01F0040EDBCF02F0050EDBCF03F08A
:101D6000060EDBCF04F0056A0450055C14E2055052
:101D70000324066E0650E56E62EC11F0066EE12A51
:101D800006C0E5FF00C0E9FF01C0F3FF025094EC7C
:101D900011F0052AE9D70450E4CF06F0E4CF05F0AE
:101DA000E4CF04F0E4CF03F0E4CF02F0E4CF01F09D
:101DB000E4CF00F0E4CFD9FF1200D9CFE5FFE1CFA7
:101DC000D9FF800EE56E0BEC11F0E12A010E706E6A
:101DD000AE0E716E050E726E200E736E779E779C3E
:101DE000040E606E0F01506B0F01006B0F01016B51
:101DF0000F01046B0F01056B0F01086B0F01096BDD
:101E00000F010C6B0F010D6B0F01106B0F01116BAC
:101E10000F01146B0F01156B0F01186B0F01196B7C
:101E20000F0119970F011C6B0F011D6B0F011D97FF
:101E3000000EE56E0BEC11F0E12AE4CFD9FF1200A1
:101E4000D9CFE5FFE1CFD9FF00C0E5FF01C0E5FF35
:101E500002C0E5FF006E020EDBCF01F0030EDBCF08
:101E600002F0AC6AAB6A00B0AC8800A202D0AC8CC5
:101E7000AB8C00A401D0AC8E00A602D0AB8801D000
:101E8000AB8A00A802D0AC8401D0AC949E9800AC80
:101E900002D09D8A01D09D9A9E9A00AE02D09D8864
:101EA00001D09D980250B06E0150AF6E949C948EFC
:101EB000AC8AAB8EE4CF02F0E4CF01F0E4CF00F0C7
:101EC000E4CFD9FF1200E8CFE5FFD8CFE5FFE0CFA0
:101ED000E5FFF3CFE5FFF4CFE5FFE9CFE5FFEACF7C
:101EE000E5FFFACFE5FFFBCFE5FFD9CFE5FFE1CF77
:101EF000D9FF00C0E5FF006AF2B4002A0050010AD1
:101F000003E1AEEC11F0F294E4CF00F0E4CFD9FF9E
:101F1000E4CFFBFFE4CFFAFFE4CFEAFFE4CFE9FF31
:101F2000E4CFF4FFE4CFF3FFE4CFE0FFE4CFD8FF4A
:101F3000E4CFE8FF1000D9CFE5FFE1CFD9FF00C023
:101F4000E5FF020EDBCF00F0030EDBCFA8FF00C0E1
:101F5000A9FFA69EA69CA684F29E550EA76EAA0E69
:101F6000A76EA682A6A202D00000FCD7A6A613D018
:101F7000450EA6EC11F0D8EC11F0006E0050FBE11C
:101F8000520EA6EC11F0D8EC11F0006E0050FBE1FF
:101F9000520EA6EC11F0A694F28EE4CF00F0E4CF3E
:101FA000D9FF1200D9CFE5FFE1CFD9FF00C0E5FF8F
:101FB00001C0E5FF02C0E5FF03C0E5FFDDEC0EF068
:101FC000006A016A0150800F800F02E1050E005C7B
:101FD00010E2970E0024026E000E0120036E02C074
:101FE000E9FF03C0EAFF000EEF6E002AD8B0012A15
:101FF000E9D7F36AE86AE4CF03F0E4CF02F0E4CF74
:1020000001F0E4CF00F0E4CFD9FF1200D9CFE5FF13
:10201000E1CFD9FF00C0E5FF01C0E5FF02C0E5FF49
:1020200003C0E5FF04C0E5FF05C0E5FF020EDBCFFE
:1020300000F0005010E1D6CF00F0016AD7CF02F0D7
:10204000036A0250056E046A0450002605500122FE
:1020500001C0F3FF0050E4CF05F0E4CF04F0E4CF7B
:1020600003F0E4CF02F0E4CF01F0E4CF00F0E4CFDE
:10207000D9FF1200D9CFE5FFE1CFD9FF00C0E5FFBE
:1020800001C0E5FF02C0E5FF03C0E5FF020EDBCFA4
:1020900000F0030EDBCF01F0040EDBCF02F00050A6
:1020A000011008E10250A6EC11F0D8EC11F0036E1B
:1020B0000350FBE10050010A02E1015001E002D0AF
:1020C00002C0C9FFE4CF03F0E4CF02F0E4CF01F097
:1020D000E4CF00F0E4CFD9FF1200D9CFE5FFE1CF84
:1020E000D9FF00C0E5FF01C0E5FF02C0E5FF020E19
:1020F000DBCF00F0030EDBCF01F00050011006E152
:102100009E9A3DEC11F0026E02500BD00050010A75
:1021100002E1015001E004D0C7A002D0C95001D0B3
:10212000E86AE4CF02F0E4CF01F0E4CF00F0E4CFBE
:10213000D9FF1200D9CFE5FFE1CFD9FF00C0E5FFFD
:1021400001C0E5FF020EDBCF00F0030EDBCF01F094
:102150000050011006E19EAA02D0010E0FD0E86ADD
:102160000DD00050010A02E1015001E006D0C7A0E5
:1021700002D0010E03D0E86A01D0E86AE4CF01F092
:10218000E4CF00F0E4CFD9FF1200D9CFE5FFE1CFD3
:10219000D9FF00C0E5FF01C0E5FF02C0E5FF03C0B5
:1021A000E5FF020EDBCF00F0030EDBCF01F00150A4
:1021B000026E036A0250D76E0050D66EE4CF03F071
:1021C000E4CF02F0E4CF01F0E4CF00F0E4CFD9FF98
:1021D0001200D9CFE5FFE1CFD9FF00C0E5FF01C074
:1021E000E5FF020EDBCF00F0030EDBCF01F0005065
:1021F000011009E1D8EC11F0006E005002E0E86A2D
:1022000003D0010E01D0E86AE4CF01F0E4CF00F082
:10221000E4CFD9FF1200D9CFE5FFE1CFD9FF00C04D
:10222000E5FF01C0E5FF020EDBCF00F01F0E6F16C9
:1022300000506F12E00E6F14016E01500018FAE1A9
:10224000E4CF01F0E4CF00F0E4CFD9FF1200E8AE14
:1022500006D0F3CFEAFFEE50EECFF3FF1200E8BC5A
:102260000BD0E9CFF6FFF3CFF7FFF86E0900F5507A
:102270000900F5CFF3FF12001200F00E0001AF15B8
:10228000AF6FABAC04D0AF91ABA001D0AF81ABA42A
:1022900002D00001AF85ABA202D00001AF87AE50E3
:1022A0001200E8AE04D0F3CFEAFFEE501200E8BC13
:1022B00008D0E9CFF6FFF3CFF7FFF86E0900F5502D
:1022C00012001200D9CFE5FFE1CFD9FF020EDBCF1C
:1022D000A9FFA69CA69EA680A850E4CFD9FF120015
:1022E000D9CFE5FFE1CFD9FFF28AF184F28EF36A0C
:1022F000010EE4CFD9FF120017EEFFF027EEFFF03A
:10230000F86AA68EA69C46EC0EF00AEC0BF0FFD7FE
:10231000E8AE07D0F3CFEAFFE4CFEEFFF4CFEEFF55
:102320001200E8AC12001200E8AE05D0F3CFEAFFCD
:10233000E4CFEEFF1200E8AC12001200617B0080D7
:1023400097008000000102030405AA00ACAC04D091
:10235000AC900001AFB3AC80AD6E1200D9CFE5FFF9
:10236000E1CFD9FFE4CFD9FF1200D9CFE5FFE1CF0C
:10237000D9FFE4CFD9FF1200D9CFE5FFE1CFD9FFD4
:10238000E4CFD9FF1200D9CFE5FFE1CFD9FFE4CFE9
:10239000D9FF1200D9CFE5FFE1CFD9FFE4CFD9FFB4
:1023A000120001003C2300007B0000001000000030
:0823B000000EACA2010F1200A7
:020000040030CA
:0E000000FFF2FFFEFFFFBBFFFFFFFFFFFFFF52
:00000001FF
